:100000000C9434000C9451000C9451000C94510049
:100010000C9451000C9451000C9451000C94FB0072
:100020000C9451000C9451000C9451000C94CA0093
:100030000C9451000C9451000C9499000C945100B4
:100040000C9451000C9451000C9451000C945100EC
:100050000C9451000C9451000C9451000C945100DC
:100060000C9451000C94510011241FBECFEFD8E026
:10007000DEBFCDBF11E0A0E0B1E0E6EAF5E002C0EE
:1000800005900D92A631B107D9F711E0A6E1B1E0D4
:1000900001C01D92AB31B107E1F70E944C010C94F5
:1000A000D1020C940000DC0154968D919C915597DF
:1000B0008230910561F08330910599F00197C9F480
:1000C00016BC80916E00826080936E0016C0109204
:1000D00085001092840080916F00826080936F0091
:1000E0000CC01092B200809170008260809370000A
:1000F00004C081E090E00E94D10278949FB7F89408
:10010000809118019FBF8823C9F31092180150965F
:10011000ED91FC91519718968D919C9119970097AC
:1001200021F4808182608083089580818D7F808327
:1001300008951F920F920FB60F9211242F933F93A1
:100140008F939F9380911601909117010196909340
:1001500017018093160180911801813091F0209150
:100160001601309117018091190190911A012817F9
:10017000390738F081E0809318011092170110922E
:1001800016019F918F913F912F910F900FBE0F906D
:100190001F9018951F920F920FB60F9211242F9354
:1001A0003F938F939F938091160190911701019631
:1001B000909317018093160180911801813091F07E
:1001C00020911601309117018091190190911A0127
:1001D0002817390738F081E0809318011092170131
:1001E000109216019F918F913F912F910F900FBE0A
:1001F0000F901F9018951F920F920FB60F92112417
:100200002F933F938F939F938091160190911701A5
:100210000196909317018093160180911801813007
:1002200091F0209116013091170180911901909160
:100230001A012817390738F081E0809318011092CD
:100240001701109216019F918F913F912F910F905E
:100250000FBE0F901F901895FC01249825E230E006
:100260003787268785B5836085BD41E050E0538B95
:10027000428B8AE090E090931A018093190184B533
:10028000826084BD89EF87BD558B448B219A318B69
:10029000208B80E090E00895CF92DF92EF92FF9262
:1002A00080E091E00E942C01C12CD12C760160E00D
:1002B00070E0CB0160930001709301018093020113
:1002C0009093030180E091E00E9453008FEFC81AE1
:1002D000D80AE80AF80AC701B6010E94E0012FE631
:1002E00032E143E05BE30E946E0220E030E0A901CE
:1002F0000E947C01DFCF5058BB27AA270ED0B4C084
:10030000A5D030F0AAD020F031F49F3F11F41EF4B4
:100310009AC00EF4E095E7FB90C0E92FB6D080F3C9
:10032000BA17620773078407950718F071F49EF5F2
:10033000CEC00EF4E0950B2EBA2FA02D0B01B90103
:1003400090010C01CA01A0011124FF27591B99F04B
:10035000593F50F4503E68F11A16F040A22F232F57
:10036000342F4427585FF3CF469537952795A795A7
:10037000F0405395C9F77EF41F16BA0B620B730B4E
:10038000840BBAF09150A1F0FF0FBB1F661F771FBF
:10039000881FC2F70EC0BA0F621F731F841F48F474
:1003A000879577956795B795F7959E3F08F0B3CFFA
:1003B0009395880F08F09927EE0F979587950895E4
:1003C000E89409C097FB3EF49095809570956195EF
:1003D0007F4F8F4F9F4F9923A9F0F92F96E9BB27A5
:1003E0009395F695879577956795B795F111F8CF21
:1003F000FAF4BB0F11F460FF1BC06F5F7F4F8F4F8C
:100400009F4F16C0882311F096E911C0772321F081
:100410009EE8872F762F05C0662371F096E8862F19
:1004200070E060E02AF09A95660F771F881FDAF770
:10043000880F9695879597F9089597F99F6780E8B3
:1004400070E060E008959FEF80EC089500240A9426
:100450001616170618060906089500240A9412169F
:100460001306140605060895092E0394000C11F4D2
:10047000882352F0BB0F40F4BF2B11F460FF04C07F
:100480006F5F7F4F8F4F9F4F089557FD9058440FD8
:10049000551F59F05F3F71F04795880F97FB991FE3
:1004A00061F09F3F79F087950895121613061406A0
:1004B000551FF2CF4695F1DF08C01616170618062D
:1004C000991FF1CF86957105610508940895E89408
:1004D000BB2766277727CB0197F908950BD0C4CFA8
:1004E000B5DF28F0BADF18F0952309F0A6CFABCF1F
:1004F0001124EECFCADFA0F3959FD1F3950F50E002
:10050000551F629FF001729FBB27F00DB11D639FC5
:10051000AA27F00DB11DAA1F649F6627B00DA11D6B
:10052000661F829F2227B00DA11D621F739FB00D11
:10053000A11D621F839FA00D611D221F749F332781
:10054000A00D611D231F849F600D211D822F762F1A
:100550006A2F11249F5750408AF0E1F088234AF017
:10056000EE0FFF1FBB1F661F771F881F9150504063
:10057000A9F79E3F510570F060CFAACF5F3FECF323
:10058000983EDCF3869577956795B795F795E7954F
:100590009F5FC1F7FE2B880F911D9695879597F960
:0605A0000895F894FFCF5E
:1005A600000000000000000000000AD7233C000005
:0605B6000000000000003F
:00000001FF
